:020000040000FA
:0A00000000000E308A00EC2E09000B
:101DC0000E308A00E02E8A010000000000000000B2
:101DD0000E308A00E02EFF3F83018B130530F800A0
:101DE0008F018E01313090000C100C1CF52E0C1060
:101DF000F80BF52E90010330860083168601FF3024
:101E0000870088008312A230ED27E727A000071A79
:101E10000E2FE727A000072FE727A0002008263A6B
:101E2000A63003199E2F8A012008223A03190028A0
:101E30000E308A002008023A031D912FE727553AF9
:101E4000031DEC2EE727003A031DEC2EE727AA3AE4
:101E5000031DEC2EE727003A031DEC2E8230ED2700
:101E6000A027A6273F308E00FF308C00C027031329
:101E7000E727F100E727F300E727F2000310F30C50
:101E8000F20C0310F30CF20CF2080319492FF30AB9
:101E90004C2FF3080319832FE7270F39F107F400BC
:101EA000E727F107F500E7273F39F107F600E727B5
:101EB000F107F7007408031D672FFC30750703183E
:101EC000672F0E30F4007508E43EF500712F0E30D8
:101ED0007402031C712F031D7C2FE0307502031860
:101EE0007C2F031774088F0075088D00A6277708CC
:101EF0008C0076088E00C02703138430ED27F20B88
:101F00004C2FF30B4C2FF1080319892F8630ED2746
:101F1000EC2EA230ED27A027A6278E018C01C0272A
:101F2000EC2EA027831680308C000C1400000000DB
:101F300083128C0803130319E32E8630ED270C2F30
:101F400003170E308F00EB308D0008000D08F500F0
:101F50000430F80021308400FC308D0583168C1786
:101F60000C140000000083120C088000840A0E0884
:101F70008000840A8D0AF80BAE2F75088D000800CA
:101F8000213084000D080339840784070C08800081
:101F9000840A0E08800021308400FC308D05000882
:101FA0008C00840A00088E00840A831684308C001A
:101FB00055308D00AA308D008C1400000000831273
:101FC0008D0A0D080339003A031DCF2F0800071AA8
:101FD000E72F8610080886140800831688018312EC
:101FE00088000610000006148316FF308800831254
:021FF0000800E7
:02400E00721F1F
:00000001FF
